:020000040000FA
:10000000012864008501860107309F0083160030B7
:100010008500003086000730810083123030900068
:100020007B3092000330A1002108BE210530A100E1
:100030000430A2002108BE21083085000630860069
:100040002108BE2108308501013086002108BE212B
:1000500004308500103086002108BE210230850062
:1000600086012108BE21013085004030860021082C
:10007000BE218501860C2108BE21860D860DA10BAF
:100080001A28A10AA20B1A28850186010A30A100AC
:100090002108BE210530A1000430A2002108BE21A4
:1000A0008501860108308500063086002108BE21C2
:1000B00006142108BE21051506162108BE21851447
:1000C0002108BE21051406172108BE218616210825
:1000D000BE2186172108BE21851186100611210830
:1000E000BE2106102108BE21051106122108BE21DD
:1000F00085102108BE21051006132108BE21861295
:100100002108BE218613A10B4E28A10AA20B4E285E
:10011000850186010A30A1002108BE210530A10019
:100120000430A2002108BE21850186012108BE21DC
:1001300006172108BE21061306152108BE21061147
:1001400005152108BE21051186172108BE21861339
:1001500086142108BE21861085142108BE21851031
:1001600085152108BE21851186162108BE2186121B
:1001700006142108BE21061005142108BE21051011
:100180000616A10B9228A10AA20B922885018601CE
:100190000530A1002108BE210F30A1000430A200CB
:1001A0002108BE21850186012108BE218509860915
:1001B000A10BD028A10AA20BD028850186010A3004
:1001C000A1002108BE210730A1000430A2002108AF
:1001D000BE21850186012108BE21851586140615DC
:1001E0002108BE218501013086002108BE210515A8
:1001F000103086002108BE210511851486012108D2
:10020000BE218510051406172108BE21051006130E
:1002100086162108BE21861286172108BE21851563
:10022000861406152108BE2185018130860021082B
:10023000BE210515061006162108BE2105118514DC
:1002400006122108BE218510051406172108BE21BB
:100250000510061386162108BE218515861406157D
:100260002108BE218501A13086002108BE21051587
:10027000061606102108BE21851405110612210854
:10028000BE218510051406172108BE218515861488
:1002900006152108BE218511E13086002108BE2106
:1002A0000515061006162108BE2105118514061233
:1002B0002108BE218515861406152108BE21851149
:1002C000E13086002108BE210515F03086002108A6
:1002D000BE218515F63086002108BE218511F1303A
:1002E00086002108BE218515F7308600A10BE7287E
:1002F000A10AA20BE728850186010A30A100210886
:10030000BE210730A1000430A2002108BE218501D2
:1003100086012108BE2186142108BE21851586107C
:1003200006152108BE218511061106142108BE21DB
:10033000051506102108BE21051106162108BE214B
:10034000851406122108BE21851005142108BE213E
:10035000061705102108BE21061386162108BE21A6
:1003600086178612A10B8529A10AA20B8529850172
:1003700086010530A1002108BE211228A000A00A94
:1003800081010B1164000B1DC229A00BC0290800BC
:02400E00143F5D
:00000001FF
